:10000000C2298C007F390C1B803C09208C1B003CD2
:1000100008008A01820700340334063409340C34A2
:1000200010341334163419341C341F34223425345C
:1000300028342B342E3431343334363439343C3490
:100040003F3441344434473449344C344E345134D1
:100050005334553458345A345C345E34603462342A
:100060006434663468346A346B346D346F3470349D
:1000700071347334743475347634783479347A3432
:100080007A347B347C347D347D347E347E347E34EB
:100090007F347F347F347F348C005E208C0073206B
:1000A00093008C0A732092008C0E732091008C0AAE
:1000B0007320882017088F0016085F2900308A00F7
:1000C0000C080F398207A6348034A034C03482343F
:1000D000A234C2348434A434C4348634C634E03404
:1000E000E234E434E63400308A000C080F39820729
:1000F0000234B93403340234033454340334AD3499
:100100000434B934053438340534C5340634613424
:10011000900011089002031C910313089202031C23
:10012000930327098E0025098F008E0A03198F0A71
:1001300041309500980199019A019B01940126088C
:100140008400240939218413BE211008980703185C
:10015000990A1108990712089A0703189B0A1308AD
:100160009B0719080120803E8D001B080120803E5E
:100170008D070D0C940700082404031C240680003E
:10018000150303194130950003198E0A03198F0FC7
:10019000A428BD299200260884000930930003108A
:1001A000D620920C930BD0280314D6288413A31DB9
:1001B000E52800082404231D240680008417000875
:1001C0002404031C24068000F02800082404031CD7
:1001D0002406231924068000841724098005F028AA
:1001E000230D06398C00F9208D008C0AF9200000BF
:1001F0006C2901308A000C080029FF3FFF3FFF3FB8
:1002000082070134993403343934003460340C34B7
:10021000FD348F00260884002409392184138F08B7
:100220000319BD29F03091000E0880389000F0309D
:1002300091030319910003198F030319BD290C08B9
:1002400092000D08930027306B2112088C001308D0
:100250008D00492103010C1824088E1F24088E08E4
:1002600003190301900F362980061429372900004D
:10027000172984178005BD2901308A001408073921
:1002800082070134023404340834103420344034FA
:1002900080340D080C0403198C0A80300C1A8D066A
:1002A0000C198D068C188D060D0D8C0D8D0DBD292C
:1002B00089008316081483120808BD298F018E0057
:1002C000FF308E07031C8F07031CBD2903308D00F0
:1002D000E6306C2160298D01FC3E8C008D09031CE9
:1002E0007729FF3000008C07031872298C076400FF
:1002F0008D0F7129080094003C218C018D01941D03
:100300008C0094198D000C08BD298C001130FF3E23
:100310008C0D8D0D031C8729BD2903108D0C8C0CB1
:10032000FF3E03188D290C08BD298E00053094006E
:100330000F080D02031D9E290E080C02043003183D
:100340000130031902301405031DFF30BD291030A0
:1003500094008D018C01930C920C031CB5290E089E
:100360008C070F0803180F0F8D078D0C8C0C910C48
:10037000900C940BAB291008BD298313031383122F
:100380006400080083160730850081138312AD01D5
:100390000508AD000330AD052D08033C031CDB2927
:1003A000D321AB00DB2901308A002D0882070734F6
:1003B000053404340634F9210530A6000430A400C5
:1003C000C830A700A50132309600970128084C20BC
:1003D0000530A6001030A40073308E000A300921C9
:1003E0000530A6000830A4002B08A3002808CA2066
:1003F000C82932305E2186018316F03086008312D0
:1004000006088C008D01043090219E000D089F008D
:100410001E088C001F088D008F010F309521031DD1
:10042000FB2932305E21AC01640004302C02031839
:10043000312A86012C087B219E000D089F00FF3089
:100440001E0683168600831206088C008D01043078
:100450009021A900640029080F3C031D322AAC0F2B
:10046000142A132A2C089200930104308E008F0165
:10047000A7219E0011089F000F302906A000003020
:10048000A10021088D0020088521A000A1011E08DF
:10049000A0071F080318013EA1072003AA002A088D
:1004A0005821A80008006300532AFF3FFF3FFF3F89
:1004B000FF3FFF3FFF3FFF3FFF3FFF3FFF3FFF3F4C
:1004C000FF3FFF3FFF3FFF3FFF3FFF3FFF3FFF3F3C
:1004D000FF3FFF3FFF3FFF3FFF3FFF3FFF3FFF3F2C
:1004E000FF3FFF3FFF3FFF3FFF3FFF3FFF3FFF3F1C
:02400E00F23F7F
:104200000100020003000F000400050006000E007C
:104210000700080009000D000A0000000B000C0058
:10422000FF00FF00FF00FF00FF00FF00FF00FF0096
:10423000FF00FF00FF00FF00FF00FF00FF00FF0086
:10424000FF00FF00FF00FF00FF00FF00FF00FF0076
:10425000FF00FF00FF00FF00FF00FF00FF00FF0066
:10426000FF00FF00FF00FF00FF00FF00FF00FF0056
:10427000FF00FF00FF00FF00FF00FF00FF00FF0046
:00000001FF
